:020000040800F2
:1000000000040020E1010008E3010008E20100080B
:10001000E2010008E2010008E2010008E201000834
:10002000E2010008E2010008E2010008D52C000806
:10003000E2010008E2010008E2010008E201000814
:10004000E2010008E2010008E2010008E201000804
:10005000E2010008E2010008352F0008612F0008C6
:100060008D2F0008B92F0008E52F0008E2010008D5
:10007000E2010008E2010008E2010008E2010008D4
:10008000E2010008E2010008E2010008E2010008C4
:10009000E2010008E2010008E20100081130000856
:1000A000E2010008E2010008E2010008E2010008A4
:1000B000512D0008E2010008E2010008E2010008F9
:1000C000E2010008E2010008E2010008E201000884
:1000D000E2010008E2010008E2010008E201000874
:1000E00079300008E2010008E2010008E20100089E
:1000F000E2010008E2010008E2010008E201000854
:10010000E2010008E2010008E2010008E201000843
:10011000E2010008E2010008E2010008E201000833
:10012000E2010008E2010008E2010008E201000823
:10013000E2010008E2010008E2010008E201000813
:10014000E2010008E2010008E2010008DD230008E6
:10015000E2010008E2010008E2010008E2010008F3
:10016000E2010008E2010008E2010008E2010008E3
:10017000E2010008E2010008E2010008E2010008D3
:10018000E2010008E2010008E2010008E2010008C3
:10019000E2010008E2010008E2010008E2010008B3
:1001A000E2010008E2010008E2010008E2010008A3
:1001B000E2010008E2010008E2010008E201000893
:1001C000E2010008E2010008E2010008E201000883
:1001D000E2010008E2010008E2010008E201000873
:1001E00002E000F000F8FEE772B6394880F30888B4
:1001F000384880F3098838484EF60851CEF200019D
:10020000086040F20000CCF200004EF63471CEF2ED
:1002100000010860BFF34F8FBFF36F8F40F2000003
:10022000C0F2F0004EF68851CEF200010860BFF334
:100230004F8FBFF36F8F4FF00000E1EE100A4EF6C4
:100240003C71CEF200010860062080F31488BFF3F1
:100250006F8F01F08FFD02F0D5FC4FF055301F4934
:100260001B4A91423CBF41F8040BFAE71C49194A6A
:1002700091423CBF41F8040BFAE71A491A4A1B4B5A
:100280009A423EBF51F8040B42F8040BF8E70020F5
:100290001749184A91423CBF41F8040BFAE701F0B4
:1002A0006DFD02F00BFD144C144DAC4203DA54F812
:1002B000041B8847F9E700F03FF8114C114DAC42A0
:1002C00003DA54F8041B8847F9E701F055BD000034
:1002D000000400200024002000000008000000208E
:1002E00000040020A8340008002400202824002056
:1002F00028240020E8330020E0010008E001000885
:10030000E0010008E00100082DE9F04F2DED108A12
:10031000C1F80CD0C3689D46BDEC108ABDE8F08FD3
:10032000002383F311882846A047002001F0F0F94C
:1003300001F0A0F900DFFEE738B5174B7D2200245D
:100340001A700F225C709C70DC701C715C719C7167
:10035000DC711C725C729A72DC7201F0EBFC0F4B68
:10036000984217D00133984241F2883412BF0025D9
:1003700000240125002001F0E3FC0DB100F052F84B
:1003800000F070FC00F030FB204600F09FF800F019
:1003900049F8F9E72546EDE728240020010007B0D9
:1003A00008B500F0C3FAA0F120035842584108BD37
:1003B00007B5054B02211B88ADF8043001A800F0F9
:1003C00003FB03B05DF804FB7431000810B511485D
:1003D000C3680BB101F022FA0F4C104A0D480023FC
:1003E0004FF47A7101F0DEF9236813B12368013B01
:1003F0002360636813B16368013B6360084B1B783B
:1004000033B9636823B9022000F0DCFB3223636058
:1004100010BD00BF342400204C290020CD0300086B
:100420004824002038B5224C236801333ED0214DAA
:10043000214B2A689A4239D9204B9B6803F100630B
:1004400003F580339A4231D2002000F0E7FA1C4BCA
:100450000220187000F0A4FB1A4B1A6C00221A64D8
:10046000196E1A66196E596C5A64596E5A665A6E2C
:100470005A6942F080025A615A6922F080025A6138
:100480005A691A6942F000521A611A6922F0005240
:100490001A611B6972B60C4B1C6023682A68202104
:1004A00081F311889D4683F30888104738BD00BF4B
:1004B0000000010804000108FFFF000828240020B4
:1004C000482400200038024008ED00E02DE9F04FFC
:1004D000B34B8246B3489C680022C2608FB0202292
:1004E00082F31188C26800930AB101F097F90023E2
:1004F000AD4AAC484FF47A7101F054F9002383F30C
:100500001188DFF8C0B2BAF1000F01D0CBF800A01B
:10051000A64FCBF8043000253B702E464FF0FF3835
:10052000012000F03DFBBAF1000F00F0C181DBF8C3
:100530000030002B40F0BC810FB0BDE8F08F0220EE
:10054000FFF72EFF002840F0AF81994B1B88ADF8D4
:100550002430022109A800F037FAE1E74FF47A705D
:1005600000F0E4F9031E0193EFDB0220FFF718FF10
:1005700081460028E9D0019B581E0428E5D8DFE811
:1005800000F00310131619000EA8052340F8143DBF
:10059000042100F019FA4D4600F05AFBFFF708FF5E
:1005A0007FE104217E48F4E704218248F1E7042139
:1005B0008148EEE71C25284600F032FA0435099000
:1005C000042109A800F000FA2C2DF4D1E3E7002E55
:1005D000BBD0002DB9D00220FFF7E2FE064610B9CD
:1005E00001252E46B1E7012000F018FA02203870EC
:1005F00000F0D6FA00255FFA85F9484600F026FAA1
:100600000135044618B1484600F030FAF3E70123FB
:1006100002203B7000F0B2FA009B9B689C4207D21C
:10062000204600F0FDF9013040F040810434F3E74A
:1006300000243C70CBF804403546ADE7002E84D052
:10064000002D82D00220387000F0AAFA322000F08B
:100650006DF9051EC4DB15F00306C1D1009A92683E
:1006600063199342BCD8B5F5807FB9D8DFF84C91B7
:10067000AE420CDA4FF47A7000F058F90390039B05
:10068000002BADDB039B06F809300136F0E7C820EC
:10069000FFF786FE06460028A2D02CB9474B4FF044
:1006A000FF32D3F800801A60444B25F0030525443F
:1006B000A3EB0409AC42BFD059F80410204600F067
:1006C000B5F9204600F0ACF959F80430984240F0F2
:1006D000ED800434EEE70220FFF762FE00283FF4CD
:1006E00034AF4FF0000AD146009B9B689A4537D241
:1006F000BAF1000F17D1B8F1FF3F14D0CDF8248024
:100700002F494B68A3B1002209A8135C83EA0903AF
:10071000DBB2013251F82330042A83EA1929F4D1DB
:100720000AF1040AE0E7504600F07AF90990E7E799
:100730001A46082012F0010F4FEA52021FBF82F042
:100740006D4282F4380282F4034282F020020138C2
:10075000F0D141F823200133B3F5807FE8D1D2E70F
:100760000EA8042140F8289D00F02EF914E70EA8E9
:10077000002340F8143D642100F002F900287FF4C2
:10078000E4AE0220FFF70CFE00283FF4DEAE09982D
:1007900000F07EF90EAB43F8240D04211846E3E780
:1007A0002824002034240020CD0300084824002001
:1007B000763100082C240020302400204C24002016
:1007C0004C2500204C2900200EA8002340F8143DA1
:1007D000642100F0D5F800287FF4B7AE0220FFF7BF
:1007E000DFFD00283FF4B1AE099800F05FF90EABD1
:1007F00043F8200DD1E70220FFF7D2FD00283FF497
:10080000A4AE00F059F90EAB43F81C0DC5E7022069
:10081000FFF7C6FD00283FF498AE09A9142000F0A8
:1008200051F981460EA8042140F8189D00F0CCF83B
:10083000494609A898E74FF47A70FFF7B1FD002800
:100840003FF483AEB8F1FF3F05D1FFF7B1FD354866
:1008500000F064FF70E64146002000F0E7F8002059
:1008600000F0DEF88045F0D02F4B6FE60EA8002395
:1008700040F8143D642100F083F800287FF465AE51
:100880000220FFF78DFD00283FF45FAEFFF790FDDB
:1008900041F2883000F042FF099800F00DFA00F0B4
:1008A000D7F94FF0000A3BE6064675E63546DBE72A
:1008B000002000F03BF80390039B002BFFF633AEC3
:1008C000012000F05BF9039B213B122B3FF628AE81
:1008D00001A252F823F000BF3F0500085D050008A3
:1008E000CF050008210500082105000821050008A2
:1008F0003D06000821050008D70600086F0700081C
:10090000C9070008F7070008210500080F080008BC
:10091000210500083708000899050008210500088E
:100920006D080008A08601007831000837B5114B2A
:100930001A780132D2B20024012A01468DF807400C
:1009400011D80D4803681D6A4FF47A734B43012296
:100950000DF10701A847012805D1084B9DF80700B4
:100960001C7003B030BD4FF4FA7000F0D7FE4FF0AA
:10097000FF30F6E7002400209C29002058290020A1
:1009800038B50E4B1A780132D2B2012A05460ED87C
:100990000B4803681C6A4FF47A734B4304222946C0
:1009A000A047042803D1074B0020187038BD4FF42E
:1009B000FA7000F0B3FE4FF0FF3038BD0024002085
:1009C0009C2900205829002030B4054C2368DD699B
:1009D000044B0A46AC460146204630BC604700BF87
:1009E0009C290020A086010070B501F0DFF8094CB9
:1009F000094E2070002530682378834208D901F021
:100A0000CFF8336805440133B5F5803F3360F2D346
:100A100070BD00BF592900205429002001F076B98B
:100A200000F1006000F580300068704707B502AB48
:100A300000F1006043F8041D0422194600F58030DF
:100A400001F0F2F803B05DF804FB0000054B1A68F2
:100A5000054B1B781344834202D9104401F0A0B81F
:100A600000207047542900205929002038B5074D2F
:100A700004462868204401F09BF828B928682044DF
:100A8000BDE8384001F0ACB838BD00BF54290020A3
:100A900010F0030308D1B0F5007F05D800F1005035
:100AA000A0F508400068704700207047014BC0580F
:100AB000704700BF107AFF1F014B1868704700BFD6
:100AC000002004E070B52A4B1C68C4F30B03240C0F
:100AD00063B140F21342934231D040F21942934243
:100AE0002FD040F2214293422DD10323214A0C25DD
:100AF00005FB03235D6893F9082042F201039C4241
:100B000024D0B4F5805F23D041F201039C4221D070
:100B100041F203039C421FD041F207039C4208BFED
:100B20003122441E0C44013D0B46A3421ED215F94E
:100B3000016F581C96B1034600F8016CF5E70123DC
:100B4000D4E70223D2E73F220B4DD6E73322E3E777
:100B50004122E1E75A22E4E75922E2E72C258442C8
:100B60001D7001D9981C5A70401A70BD1846FBE7D9
:100B7000002004E0883100087C310008022804D1FC
:100B8000054B4FF000729A6170470128FCD14FF07D
:100B90008042024BF7E700BF000402400000024021
:100BA000022804D1054B4FF400729A617047012866
:100BB000FCD14FF48042024BF7E700BF0004024033
:100BC00000000240022805D1064A536983F40073ED
:100BD000536170470128FCD1034A536983F4804371
:100BE000F6E700BF000402400000024010B50023F9
:100BF000934203D0CC5CC4540133F9E710BD00002C
:100C000030B5441E14F9010F0B4660B193F9005042
:100C1000854201F1010106D11AB993F90020801A29
:100C200030BD013AEEE7002AF7D1104630BD000092
:100C300002460346981A13F9011B0029FAD170479E
:100C400002440346934202D003F8011BFAE77047BF
:100C5000024B1A78024B1A70704700BF58290020C7
:100C60000024002038B5104D104C284600F0A4F8A0
:100C70002146284600F0CCF823680D485A6DD2F87A
:100C8000043843F00203C2F8043800F047FD094974
:100C9000206800F0C3F923685A6DD2F8043823F0B5
:100CA0000203C2F8043838BD9C29002054320008E1
:100CB00040420F00A43200087047000002684368F9
:100CC0001143016003B118477047000013B5446B2E
:100CD000D4F894341A681178042916D1217C022999
:100CE00013D11979128901238B4013420DD101A927
:100CF00004F14C0001F0EAFD024630B1D4F894440E
:100D0000019B2179206800F0D5F902B010BD0000E8
:100D1000143001F059BD00004FF0FF33143001F0E2
:100D200053BD00004C3001F03DBE00004FF0FF33DA
:100D30004C3001F037BE0000143001F027BD000038
:100D40004FF0FF31143001F021BD00004C3001F0B4
:100D500009BE00004FF0FF324C3001F003BE00002E
:100D6000D0F8942438B5136819780429054601D0C1
:100D7000012038BD017C0229FAD112795C89012059
:100D800090400440F4D105F1140001F0B9FC024692
:100D90000028EDD0D5F894544FF480732868697911
:100DA00000F076F9204638BD406BFFF7D9BF000050
:100DB00000207047704700007FB5124B036000238E
:100DC00043608360C360012502260F4B057404460F
:100DD0000290019300F18402294600964FF480733B
:100DE000143001F069FC094B0193029400964FF412
:100DF000807304F52372294604F14C0001F042FD92
:100E000004B070BDD8310008A90D0008CD0C000851
:100E10000B68202282F311880A7903EB8202906129
:100E20004A79093243F822008A7912B103EB82032E
:100E3000986102230374C0F89414002383F311888B
:100E40007047000038B50446012502210430FFF741
:100E500035FF04F1140025776FF0010100F086FCE6
:100E600084F8545004F14C006FF00101BDE83840A3
:100E700000F07CBC10B5012104460430FFF71EFFD2
:100E80000023237784F8543010BD000038B50446A1
:100E90000025143001F028FC04F14C00257701F006
:100EA00009FD201D84F854500121FFF707FF20465B
:100EB000BDE83840FFF754BF90F8443003F06003BA
:100EC000202B19D190F84520212A0AD0222A4FF050
:100ED00000030ED0202A0FD1084A82630722C26382
:100EE00004E0064B83630723C363002303640120EC
:100EF00070478363C363F9E7002070470124002033
:100F0000D0F8943437B51A681178042904461AD1F8
:100F1000017C022917D11979128901238B401342D0
:100F200011D100F14C05284601F09AFD58B101A9F4
:100F3000284601F0CBFCD4F89444019B2179024669
:100F4000206800F0B7F803B030BD000000EB81036B
:100F5000F7B59C6905460E46F4B1202383F311884A
:100F600005EB8607201D0821FFF7A8FEFB685B69DB
:100F70001B684C3413B1204601F0B6FC01A9204691
:100F800001F0A4FC024648B1019B3146284600F01E
:100F900091F8002383F3118803B0F0BDFB685A6910
:100FA0001268002AF5D01B8A013B1340F1D105F1EC
:100FB0004402EAE7093138B550F82140DCB120237A
:100FC00083F31188D4F894241368527903EB8203D5
:100FD000DB689B695D6845B104216018FFF76EFE10
:100FE000294604F1140001F095FB2046FFF7B8FEF6
:100FF000002383F3118838BD7047000000F044BF20
:101000000123037000234360C36183620362C362F0
:1010100043620363038143817047000038B504468F
:10102000202383F3118800254160C5600561456177
:10103000856100F039FF0223237085F3118838BDE4
:1010400070B500EB810305465069DA600E46144620
:1010500018B110220021FFF7F3FDA06918B110228A
:101060000021FFF7EDFD31462846BDE8704000F055
:10107000E1BF0000028902F001020281428902F010
:1010800001024281002202614261826101F066B880
:10109000F0B400EB81044789E4680125A4698D4020
:1010A0003D43458123600023A2606360F0BC01F0F2
:1010B00081B80000F0B400EB81040789E4680125E1
:1010C00064698D403D43058123600023A260636015
:1010D000F0BC01F0FBB8000070B502230025044607
:1010E0000370A0F84C5080F84E5080F84F500581A6
:1010F0004581C56005614561856180F8345000F027
:1011000035FF63681B6823B129462046BDE870405F
:10111000184770BD436802781B6880F8502005228C
:1011200002700BB10421184770470000436890F823
:1011300050201B6802700BB1052118477047000052
:1011400090F8343070B5044613B1002380F8343081
:1011500004F14402204601F023F863689B6863BBF6
:1011600094F8445015F0600615D194F8453005F018
:101170007F0545EA032540F202339D4200F00E81CF
:101180005BD8022D00F0DC803FD8002D00F0878076
:10119000012D00F0CF800021204601F059FA0021F6
:1011A000204601F04BFA63681B6813B10621204604
:1011B0009847062384F8343070BD204698470028AD
:1011C000CED094F84B2094F84A3043EA0223E26BE5
:1011D000934238BFE36394F94430E56B002B4FF042
:1011E000200380F2FD80002D00F0EC80092284F8BD
:1011F000342083F311880021E36BA26B2046FFF7B4
:1012000059FF002383F3118870BDB5F5817F00F08D
:10121000B180B5F5407F49D0B5F5807FBBD194F85A
:101220004630012BB7D1B4F84C3023F00203A4F8B8
:101230004C30A663E6632664C3E740F201639D4237
:101240001ED8B5F5C06F3BD2B5F5A06FA3D1B4F8E9
:101250004430B3F5A06F0ED194F8463084F84E3088
:10126000204600F0DBFE63681B6813B101212046B5
:101270009847032323700023A363E3632364A0E759
:10128000B5F5106F32D040F602439D4252D0B5F50D
:10129000006F80D104F14F03A363012324E004F124
:1012A0004C03A3630223E36325648AE794F8463082
:1012B000012B7FF470AFB4F84C3043F00203B6E773
:1012C00094F84920616894F848304D6894F84710C4
:1012D00043EA0223204694F84620A84700283FF41A
:1012E0005AAF4368A3630368E363A4E72378042B3E
:1012F00010D1202383F311882046FFF7BBFE86F32D
:101300001188636884F84F601B68032121700BB15A
:101310002046984794F84630002BACD084F84F30E4
:101320000423237063681B68002BA4D0022120468D
:101330009847A0E7374BA3630223E36300239DE7AD
:1013400094F8481011F0800F204601F00F010ED0E4
:1013500000F018FF012806D002287FF41CAF2E4BA6
:10136000A363E06367E72D4BA363E56363E700F0E6
:10137000FBFEEFE794F84630002B7FF40CAF94F8B7
:10138000483013F00F013FF476AF1A06204602D51D
:1013900001F072F96FE701F065F96CE794F84630F7
:1013A000002B7FF4F8AE94F8483013F00F013FF4AF
:1013B00062AF1B06204602D501F04AF95BE701F057
:1013C0003DF958E7142284F8342083F311882B4622
:1013D0002A4629462046FFF75BFE85F3118870BD3B
:1013E0005DB1152284F8342083F311880021E36B6A
:1013F000A26B2046FFF74CFE03E70B2284F8342053
:1014000083F311882B462A4629462046FFF752FED1
:10141000E3E700BF08320008003200080432000889
:1014200038B590F834300446152B29D8DFE803F09E
:101430003E28282828283E28280B2939282828280B
:10144000282828283E3E90F84B1090F84A20C36B7D
:1014500042EA01229A4214D9C268128AB3FBF2F519
:1014600002FB15356DB9202383F311882B462A46DC
:101470002946FFF71FFE85F311880A2384F83430CC
:1014800038BD142384F83430202383F311880023DB
:101490001A4619462046FFF7FBFD002383F3118807
:1014A00038BD036C03B198470023E7E7002101F042
:1014B000CFF80021204601F0C1F863681B6813B122
:1014C0000621204698470623D8E7000090F83420EC
:1014D000152A38B5044622D80123934040F64162CC
:1014E00013421DD113F480150FD19B0217D50B2386
:1014F00080F83430202383F311882B462A4629466E
:10150000FFF7D8FD85F3118838BDC3689B695B6818
:101510002BB9036C03B19847002384F8343038BDED
:10152000002101F095F80021204601F087F863685A
:101530001B6813B10621204698470623EDE70000FB
:10154000024B00221B605B609A6070475C290020A0
:10155000002303748268054B1B6899689142FBD293
:101560005A68036042601060586070475C29002030
:1015700008B5202383F31188037C032B05D0042BAB
:101580000DD02BB983F3118808BD436900221A607E
:101590004FF0FF334361FFF7DBFF0023F2E790E8F2
:1015A0000C001A6002685360F2E700000023037425
:1015B0008268054B1B6899689142FBD85A680360A2
:1015C00042601060586070475C290020054B196923
:1015D0000874186802681A60536018610123037464
:1015E000FEF792BE5C29002030B54B1C87B0054643
:1015F0000A4C10D023690A4A01A800F0D3F8284603
:10160000FFF7E4FF049B13B101A800F007F9236979
:10161000586907B030BDFFF7D9FFF8E75C29002013
:101620007115000838B50C4D41612B6981689A68C5
:101630009142044603D8BDE83840FFF789BF1846F9
:10164000FFF786FF01232C61014623742046BDE885
:101650003840FEF759BE00BF5C290020044B1A68D1
:101660001B6990689B68984294BF002001207047D6
:101670005C29002010B5084C236820691A68226094
:101680005460012223611A74FFF790FF014620691C
:10169000BDE81040FEF738BE5C29002082600222BF
:1016A00002740022427470478368A3F17C0243F8FD
:1016B0000C2C026943F83C2C426943F8382C074A49
:1016C00043F81C2CC26843F8102C022203F8082CA3
:1016D000002203F8072CA3F118007047210300082B
:1016E00010B5202383F31188FFF7DEFF00210446A5
:1016F000FFF798FF002383F31188204610BD0000F8
:10170000024B1B6958610F20FFF760BF5C29002066
:10171000202383F31188FFF7F3BF000008B50146CB
:10172000202383F311880820FFF75EFF002383F353
:10173000118808BD49B1064B42681B6918605A60A0
:10174000136043600420FFF74FBF4FF0FF30704736
:101750005C2900200368984206D01A680260506035
:1017600059611846FFF7F4BE7047000038B50446CB
:101770000D462068844200D138BD036823605C6058
:101780004561FFF7E5FEF4E7054B03F114025A61EA
:101790009A614FF0FF32DA6100221A62704700BF8F
:1017A0005C290020F8B503614FF08043C2605C6A99
:1017B000194B1A46022952F8145F38BF022195428C
:1017C00006461F460AD1586198611C620560456053
:1017D00081600819BDE8F84001F064B9186AAB6887
:1017E000241A0C1902D3E41A2D6804E09C4202D298
:1017F000204401F065F9AB689C42F4D86B687360D3
:1018000035601E606E60B460A9684FF0FF33091B3D
:10181000A960FB61F8BD00BF5C29002010B41B4C1F
:10182000234653F8141F814210D0416802680A60B1
:10183000026851609A424FF00001C16003D0936882
:1018400081680B4493605DF8044B70470A686261DD
:1018500000209A425360C86003D15DF8044B01F048
:1018600029B993688868034493604FF08042206AE6
:10187000526A121A9342E6D9991A012998BF931C09
:1018800018445DF8044B01F01BB900BF5C2900202F
:1018900000207047FEE70000704700004FF0FF3067
:1018A00070470000022906D0032906D00129064806
:1018B00018BF0020704705487047032A9ABF0448A4
:1018C00000EBC2000020704700330008B43200086B
:1018D0000824002070B5044608460D46FFF7A8F915
:1018E000C6B22046013403780BB9184670BD3246A3
:1018F0002946FFF785F90028F3D1012070BD0000CB
:101900002DE9F04F80469BB008460C461646FFF77F
:101910008FF93C49C5B22046FFF7DCFF08B1063518
:10192000EDB239492046FFF7D5FF08B11035EDB2C9
:10193000632D01AF0CD8DFF8DC90DFF8DCB03D465A
:1019400094F800A0BAF1000F1CD185F800A003E0C4
:101950002146384601F006FC3846FFF769F9C0B267
:10196000431C5B0088E84800337003237370002336
:1019700002361946DAB2904206F102063BD81BB095
:10198000BDE8F08FBAF1250F30D107221D4920465E
:10199000FFF736F970B91D4B2A4603F10C0153F8D5
:1019A000040B42F8040B8B42F9D11B7813700734F7
:1019B0000D35C5E7082214492046FFF721F9A8B9DB
:1019C0001349AB1C11F8012F100902F00F0210F897
:1019D000090012F8092003F8020C594503F8012CFC
:1019E00003F10203EED118350834A9E785F800A009
:1019F00001340135A4E7FA5C06F8022C06F8011C54
:101A00000133B7E75C320008643200086D32000829
:101A10000F7AFF1F7B3200081B7AFF1F08B52023B7
:101A200083F311880348FFF76BFA002383F31188CF
:101A300008BD00BF9C29002010B50446052916D812
:101A4000DFE801F016150316161D202383F3118815
:101A50000E4A0121FFF7F4FA20460D4A0221FFF752
:101A6000EFFA0C48FFF712FA002383F3118810BD38
:101A7000202383F311880748FFF7E4F9F4E72023D4
:101A800083F311880348FFF7F5F9EDE70C320008FE
:101A9000303200089C29002038B50C4D0C4C0D4903
:101AA0002A4604F10800FFF72BFF05F1CA0204F1F2
:101AB00010000949FFF724FF05F5CA7204F1180068
:101AC0000649BDE83840FFF71BBF00BF642E002069
:101AD000082400208C320008963200086432000886
:101AE000BFF34F8F024AD368DB03FCD4704700BFBB
:101AF000003C024008B5094B1B7873B9FFF7F0FFB3
:101B0000074B1A69002ABFBF064A5A6002F18832A1
:101B10005A601A6822F480621A6008BDC230002040
:101B2000003C02402301674508B50B4B1B7893B975
:101B3000FFF7D6FF094B1A6942F000421A611A6892
:101B400042F480521A601A6822F480521A601A68AD
:101B500042F480621A6008BDC2300020003C02409E
:101B60000B2870B513D80B4A0B4C137863B90B4E86
:101B70004FF0006144F8231056F8235001330C2B2A
:101B80002944F7D10123137054F8200070BD0020C0
:101B900070BD00BFF4300020C430002020330008A6
:101BA000014B53F820007047203300080C20704789
:101BB0000B2810B5044601D9002010BDFFF7D0FF57
:101BC000064B53F824301844C21A0BB9012010BD3B
:101BD00012680132F0D1043BF6E700BF2033000861
:101BE0000B2808B51BD8FFF77BFFFFF783FF0D49D4
:101BF000F323CB60FFF774FFC300DBB243F4007341
:101C000043F002030B610B6943F480330B61FFF770
:101C100067FFFFF789FFBDE80840FFF7C9BF002055
:101C200008BD00BF003C02402DE9F047D40715462F
:101C30004DD41318B3F1016F49D2324B1B68DA0748
:101C400045D5314CFFF756FFF323E360FFF748FF1C
:101C50002F46401A40F20129032F884601EB000667
:101C600018D8294C40F201197B1A4344012B01EB8F
:101C7000000623692FD823F001032361FFF754FFE7
:101C80002846BDE8F087366851F8043CB34218D1C5
:101C9000043FE1E7B307E4D1236923F440732361F0
:101CA000236943EA090323610431D8F80030336023
:101CB000BFF34F8FFFF714FFE368002BE3D0F3234C
:101CC000E360236923F001032361FFF72DFF4FF049
:101CD000FF30BDE8F08723F440732361236943EAB2
:101CE000090323618A4631F8023B3380BFF34F8FEB
:101CF000FFF7F6FE3688BAF80030B6B2B342B3D07A
:101D0000DFE700BF00380240003C0240084908B548
:101D10000B7828B153B9FFF7EDFE01230B7008BD16
:101D200023B1BDE808400870FFF7FEBE08BD00BF44
:101D3000C2300020014B186D704700BF00280040E2
:101D4000094B1A6F120407D41A6F42F400721A6713
:101D50001A6F42F400421A67044A136843F480730E
:101D60001360034B18657047003802400070004054
:101D70000028004070470000FEE70000084A094BB9
:101D800009498B4204D3094A0021934205D3704785
:101D900052F8040F43F8040BF3E743F8041BF4E78D
:101DA000CC340008E8330020E8330020E83300207A
:101DB000836D30B500229D68446D11464FF0FF30B1
:101DC00004EB421301329542C3F80019C3F810190D
:101DD000C3F80809C3F8001BC3F8101BC3F8080BAD
:101DE000EED24FF00113C4F81C3830BD890141F028
:101DF0002001016103699B06FCD4122000F0E8BEBB
:101E0000204B03EB80022DE9F047D2F80CE05D6D2A
:101E1000DEF81420461CD2F800C005EB063605EBB0
:101E20004018516861450BD3D5F83428012303FAD3
:101E300000F022EA0000C5F834081846BDE8F08733
:101E4000BEF81040ACEB0103A34228BF2346D8F8EC
:101E50001849A4B2B3EB840F10D894681F46A4F1BC
:101E6000040959F804AFC6F800A0042F01D9043FB3
:101E7000F7E71C440B4494605360D2E70020BDE8B0
:101E8000F08700BFF830002010B5054C2046FFF762
:101E9000B7F84FF0A0436365024BA36510BD00BFC8
:101EA000F8300020743300080378012B70B5054624
:101EB0004DD1284B446D98421BD1274B5A6B42F0B1
:101EC00080025A635A6D42F080025A655A6D5A690F
:101ED00042F080025A615A6922F080025A610E2152
:101EE00043205B6900F0D2FB1C4BE3601C4BC4F841
:101EF00000380023C4F8003EC02323604FF40413CD
:101F0000A3636E6D202000F063FE0123336133690B
:101F1000DB07FCD4122000F05BFE3369002BFCDAF7
:101F20000026A6602846FFF743FF6B68C4F81068D8
:101F3000DB68C4F81468C4F81C684BB9094BA3618A
:101F40004FF0FF336361A36843F00103A36070BDEA
:101F5000054BF4E7F8300020003802404014004000
:101F600003002002003C30C0083C30C0F8B5446D8E
:101F7000054600212046FFF739FFA96D00234FF0E9
:101F800001128F68C4F834384FF00066C4F81C287A
:101F90004FF0FF3004EB431201339F42C2F8006957
:101FA000C2F8006BC2F80809C2F8080BF2D20B683D
:101FB0006A6DEB65636210231361166916F01006F3
:101FC000FBD1122000F004FED4F8003823F4FE63A5
:101FD000C4F80038A36943F4402343F01003A3611D
:101FE0000923C4F81038C4F814380A4BEB604FF0DA
:101FF000C043C4F8103B084BC4F8003BC4F8106958
:10200000C4F80039EB6D03F1100243F48013EA6564
:10201000A362F8BD5033000840800010426D90F874
:102020004E10D2F8003823F4FE6343EA0113C2F8DD
:10203000003870472DE9F0410EB200EB86080D46DE
:10204000D8F80C100F6807F00303022B50D0032BB5
:1020500050D03D4A3D4F012B18BF1746446D4FEA03
:10206000451E04EB0E030022C3F8102B8A6905F10C
:10207000100C002A40D04A8A05F158035B013A430C
:10208000E2500123D4F81C2803FA0CF31343A644AE
:102090004A69C4F81C380023CEF8103905F13F0313
:1020A000002A39D00A8A898B9208012988BF4A43BD
:1020B000C16D04EB8303561841EA0242C665294606
:1020C0005A602046FFF792FED8F80C301B8A43EA8C
:1020D00085531F4305F148035B01E7500123D4F802
:1020E0001C2803FA05F51543C4F81C58BDE8F08117
:1020F000174FB3E7174FB1E704EB4613D3F8002BA4
:1021000022F40042C3F8002BD4F81C28012303FA60
:102110000CF322EA0303BAE704EB83030E4A5A6086
:1021200004EB461629462046FFF760FED6F8003934
:1021300023F40043C6F80039D4F81C38012202FA0F
:1021400005F523EA0505CFE70080001000800410A4
:102150000080081000800C1000040002826D1268DC
:10216000C265FFF725BE00005831436D49015B5839
:1021700013F4004004D013F4001F14BF0120022008
:10218000704700004831436D49015B5813F400402B
:1021900004D013F4001F14BF012002207047000078
:1021A00000EB8101CB68196A0B6813604B685360C0
:1021B0007047000000EB810330B5DD68AA69136841
:1021C000D36019B9402B84BF402313606B8A146815
:1021D000426D1C44013CB4FBF3F46343033323F02E
:1021E000030302EB411043EAC44343F0C043C0F889
:1021F000103B2B6803F00303012B09B20ED1D2F878
:10220000083802EB411013F4807FD0F8003B14BF74
:1022100043F0805343F00053C0F8003B02EB4112FF
:10222000D2F8003B43F00443C2F8003B30BD00004D
:102230002DE9F041244D6E6D06EB40130446D3F8B2
:10224000087BC3F8087B38070AD5D6F81438190775
:1022500006D505EB84032146DB6828465B68984772
:10226000FA072FD5D6F81438DB072BD505EB8403F6
:10227000D968CCB98B69488A5E68B6FBF0F200FB7E
:1022800012628AB91868DA6890420DD2121A83E88D
:102290001400202383F311880B482146FFF78AFF9F
:1022A00084F31188BDE8F081012303FA04F26B89FD
:1022B00023EA02036B81CB6823B121460248BDE8C3
:1022C000F0411847BDE8F081F830002000EB8103B1
:1022D00070B5DD68436D6C692668E6604A0156BBDF
:1022E0001A444FF40020C2F810092A6802F00302D1
:1022F000012A0AB20ED1D3F8080803EB421410F4F5
:10230000807FD4F8000914BF40F0805040F00050A6
:10231000C4F8000903EB4212D2F8000940F004406F
:10232000C2F80009D3F83408012202FA01F101438E
:10233000C3F8341870BD19B9402E84BF4020206006
:1023400020682E8A841940F00050013C1A44B4FBE6
:10235000F6F440EAC440C6E7F8B504461E48456DA9
:1023600005EB4413D3F80869C3F80869F10717D5DA
:10237000D5F81038DA0713D500EB8403D9684B6918
:102380001F68DA68974218D2D21B00271A605F6074
:10239000202383F311882146FFF798FF87F31188E4
:1023A000330617D5D5F834280123A340134211D0A2
:1023B0002046BDE8F840FFF723BD012303FA04F2ED
:1023C000038923EA020303818B68002BE8D02146AE
:1023D0009847E5E7F8BD00BFF830002096482DE9A2
:1023E000F84F456D6E69AB691E4016F4805F6E61F3
:1023F000044605D0FEF770FEBDE8F84F00F07ABC49
:10240000002E12DAD5F8003E8B489B071EBFD5F888
:10241000003E23F00303C5F8003ED5F8043823F04E
:102420000103C5F80438FEF781FE370502D582485E
:10243000FEF770FEB0040CD5D5F8083813F0060F7F
:10244000EB6823F470530CBF43F4105343F4A053D0
:10245000EB60310704D56368DB680BB176489847B9
:10246000F2025AD4B3020CD5D4F85480DFF8C8A1D4
:1024700000274FF00109A36D9B68F9B28B4280F0F1
:102480008780F70619D5616D0A6AC2F30A1702F050
:102490000F0302F4F012B2F5802F00F0A180B2F524
:1024A000402F0AD104EB830301F58051DB68186AE1
:1024B00000231A469F4240F087803003D5F8184821
:1024C00013D5E10302D50020FFF7B2FEA20302D527
:1024D0000120FFF7ADFE630302D50220FFF7A8FE3F
:1024E000270302D50320FFF7A3FE750384D5E00779
:1024F00002D50020FFF730FFA10702D50120FFF72A
:102500002BFF620702D50220FFF726FF23077FF586
:1025100073AF0320FFF720FF6EE7D4F85480DFF895
:1025200018A100274FF00109A36D9B685FFA87FB94
:102530005B4597D308EB4B13D3F8002902F44022F4
:10254000B2F5802F22D1D3F80029002A1EDAD3F861
:10255000002942F09042C3F80029D3F80029002A4C
:10256000FBDB5946606DFFF741FC228909FA0BF34A
:1025700022EA0303238104EB8B03DB689B6813B11E
:102580005946504698475846FFF73AFC0137CBE783
:1025900008EB4112D2F8003B03F44023B3F5802F3F
:1025A00010D1D2F8003B002B0CDA628909FA01F352
:1025B00022EA0303638104EB8103DB68DB680BB170
:1025C00050469847013756E79C0708BF0A68072B13
:1025D00098BF027003F101039CBF120A013069E742
:1025E000023304EB830201F580515268906902685E
:1025F000D0F808C04068A2EB000E002210469742B7
:102600000AD104EB830463689B699A683A449A6030
:102610005A6817445F6050E712F0030F08BF08685C
:10262000964588BF8CF8000002F1010284BF000AC1
:102630000CF1010CE3E700BFF8300020436D03EB21
:102640004111D1F8003B43F40013C1F8003B70473F
:10265000436D03EB4111D1F8003943F40013C1F885
:1026600000397047436D03EB4111D1F8003B23F46F
:102670000013C1F8003B7047436D03EB4111D1F8E3
:10268000003923F40013C1F80039704700F16043AA
:1026900000F01F02400903F5614309018000C9B23F
:1026A00000F1604083F8001300F56140012393407E
:1026B000C0F880310360704730B5039C0172043369
:1026C00004FB0325C361049B03630021059B006099
:1026D0004060C16042610261856104624262816260
:1026E000C162436330BD00000022416A4161016163
:1026F000C2608262C2626FF00101FFF737B800006A
:1027000003694269934203D1C2680AB1002070474D
:10271000181D704703691960C2680132C260C2693E
:10272000134482690361934224BF436A0361002119
:10273000FFF710B838B504460D46E3683BB162694F
:10274000131D1268A3621344E362002038BD237A8C
:1027500033B929462046FEF7EDFF0028EDDA38BDF3
:102760006FF00100FBE70000C368C269013BC36072
:102770004369134482694361934224BF436A4361BE
:1027800000238362036B03B11847704770B52023A1
:10279000044683F31188866A3EB9FFF7CBFF0546EE
:1027A00018B186F31188284670BDA36AE26A13F84F
:1027B000015BA362934202D32046FFF7D5FF0023BB
:1027C00083F31188EFE700002DE9F74F1F46044619
:1027D0000E469146202383F311884FF08048002550
:1027E000D8F82430FB18009307F1FF3AAB46A36AF0
:1027F000ABB91AF1030F06D939462046FFF79AFF05
:1028000068B1002305E0D8F82410009A511A8F42CD
:10281000F3D283F31188284603B0BDE8F08FA16A94
:10282000E36AA9EB05025B1A934228BF1346402BCB
:102830001CD9334601F1400251F8040B43F8040B54
:102840009142F9D1A36A40334036A3624035A26A6F
:10285000E36A9A4202D32046FFF786FF8BF3118882
:102860004D45D8D2202383F31188C0E71A4630465D
:102870000193FEF7BBF9019BA26A1A441E44A262AF
:102880001D44E4E710B5029C0172043303FB0421EC
:10289000C36100238362C362039B0363049B0060E4
:1028A0004060C460426102618161046242624363CC
:1028B00010BD0000026AC260426A426102610022E9
:1028C0008262C2626FF00101FEF750BF4369026984
:1028D0009A4203D1C2680AB100207047184650F8E6
:1028E000043B0B6070470000C368C2690133C360DA
:1028F0004369134482694361934224BF436A43613D
:102900000021FEF727BF000038B504460D46E368F6
:102910003BB123691A1DA262E2691344E3620020FD
:1029200038BD237A33B929462046FEF703FF002835
:10293000EDDA38BD6FF00100FBE7000003691960B4
:10294000C268013AC260C26913448269036193425A
:1029500024BF436A036100238362036B03B11847FA
:102960007047000070B5202304460E4683F311889B
:10297000856A35B91146FFF7C7FF10B185F3118895
:1029800070BDA36A1E70A36AE26A01339342A36218
:1029900004D3E16920460439FFF7D0FF002080F31B
:1029A000118870BD2DE9F74F1F4604460D4691462C
:1029B000202383F311884FF080480026D8F8243074
:1029C000FB18009307F1FF3AB346A36AABB91AF1BB
:1029D000030F06D939462046FFF796FF68B100235A
:1029E00005E0D8F82410009A511A8F42F3D283F3ED
:1029F0001188304603B0BDE8F08FA06AE36AA9EB06
:102A000006021B1A934228BF1346402B1CD905F11E
:102A1000400355F8042B40F8042B9D42F9D1A36ADA
:102A20004033A3624036A26AE36A9A4204D3E16962
:102A300020460439FFF782FF8BF311884E45D8D228
:102A4000202383F31188C0E71A4629460193FEF735
:102A5000CDF8019BA26A1A441D44A2621E44E2E71B
:102A6000026943699A4203D1C3681BB9184670478B
:102A70000023FBE7836A002BF8D0043B9B1AF5D0B8
:102A80001360C368013BC360C3691A448369026170
:102A90009A4224BF436A0361002383620123E5E76E
:102AA00000F06AB94FF08043002258631A61022295
:102AB000DA6070474FF080430022DA607047000010
:102AC0004FF0804358637047FEE7000010B5174C85
:102AD000FEF736FDFEF758FE802215492046FEF728
:102AE000DDFD012344F8180C0374124B124AD96817
:102AF00021F4E0610904090C0A431049DA60CA684C
:102B000042F08072CA600E490A6842F001020A600F
:102B10001022DA77202283F82220002383F3118801
:102B200062B60848BDE81040FEF7DABD84290020EF
:102B30008033000800ED00E00003FA05F0ED00E04E
:102B4000001000E0883300082DE9F84F1F4C4FF0CB
:102B50000008656904F11407C1464FF08043266AF6
:102B60005B6AAA689E1B96421DD34FF0200AAA6892
:102B7000236AD5F80CB0134423622B68BB425F6014
:102B8000A6EB02066361C5F80C8001D1FFF792FF46
:102B900089F311882869D8478AF311886569AB6879
:102BA0009E42E4D2D9E76269BA420CD091682362AE
:102BB0008E1B9660A86802282CBF1818981CBDE8C8
:102BC000F84FFFF77DBFBDE8F88F00BF5C290020FC
:102BD000034B59685A68521A9042FBD8704700BF9D
:102BE000001000E04B6843608B688360CB68C36073
:102BF0000B6943614B6903628B6943620B68036035
:102C00007047000008B5224B22481A6940F2FF11B4
:102C10000A431A611A6922F4FF7222F001021A6152
:102C20001A691A6B0A431A631A6D0A431A651A4A1B
:102C30001B6D1146FFF7D6FF184802F11C01FFF784
:102C4000D1FF174802F13801FFF7CCFF154802F118
:102C50005401FFF7C7FF144802F17001FFF7C2FFEC
:102C6000124802F18C01FFF7BDFF114802F1A801E3
:102C7000FFF7B8FF0F4802F1C401FFF7B3FF0E489A
:102C800002F1E001FFF7AEFFBDE8084000F0DEB85A
:102C90000038024000000240A8330008000402404F
:102CA00000080240000C02400010024000140240E4
:102CB00000180240001C02400020024008B500F04D
:102CC00035FAFFF703FFBDE80840FEF7E5BE000058
:102CD00070470000064A536823F001035360EFF386
:102CE0000983683383F30988002383F311887047CD
:102CF00030EF00E010B5202383F31188104B5B68A0
:102D000013F4006318D0F1EE103AEFF309844FF09A
:102D1000807344F84C3C0B4BDB6844F8083CA4F14E
:102D2000680383F30988FEF799FC18B1064B44F851
:102D3000503C10BD054BFAE783F3118810BD00BF6E
:102D400000ED00E030EF00E031030008340300083C
:102D50004FF0804310B51A69920708D500241C6112
:102D6000202383F31188FFF7EFFE84F31188BDE879
:102D70001040FFF7BFBF0000104B1A6C42F0010279
:102D80001A641A6E42F001021A660D4A1B6E9368AD
:102D900043F0010393604FF0804353229A624FF057
:102DA000FF32DA6200229A615A63DA605A600122C5
:102DB0005A6108211A601C20FFF768BC00380240E5
:102DC000002004E01F4B1A696FEAC2526FEAD25228
:102DD0001A611A69C2F308021A614FF0FF301A69CA
:102DE0005A69586100215A6959615A691A6A62F030
:102DF00080521A621A6A02F080521A621A6A5A6A79
:102E000058625A6A59625A6A1A6C42F080521A64BD
:102E10001A6E42F080521A661A6E0B4A106840F41D
:102E200080701060186F00F44070B0F5007F1EBF16
:102E30004FF4803018671967536823F400735360A8
:102E400000F054B90038024000700040304B4FF0A1
:102E500080521A642F4A4FF4404111601A6842F0C0
:102E600001021A601A689207FCD59A6822F00302E0
:102E70009A60274B19469A6812F00C02FBD1186829
:102E800000F0F90018609A601A6842F480321A6003
:102E90000B689B03FCD54B6F43F001034B671C4B46
:102EA0005A6F9007FCD51C4A5A601A6842F080722B
:102EB0001A60184A53685904FCD5154B1A689201D8
:102EC000FCD5164A9A60164B1A68164B9A42164B56
:102ED0001BD1164A1168164A914216D140F20512CA
:102EE0001A600B4B9A6842F002029A609A6802F0EC
:102EF0000C02082AFAD15A6C42F480425A645A6E83
:102F000042F480425A665B6E704740F20572E7E712
:102F10000038024000700040085440070094883890
:102F2000002004E011640020003C024000ED00E0BD
:102F300041C20F41084A08B5536911680B4003F0BC
:102F40000103536123B1054A13680BB150689847D8
:102F5000BDE80840FFF7CEBE003C014068330020CA
:102F6000084A08B5536911680B4003F00203536126
:102F700023B1054A93680BB1D0689847BDE8084073
:102F8000FFF7B8BE003C014068330020084A08B58E
:102F9000536911680B4003F00403536123B1054AE0
:102FA00013690BB150699847BDE80840FFF7A2BE0E
:102FB000003C014068330020084A08B55369116895
:102FC0000B4003F00803536123B1054A93690BB129
:102FD000D0699847BDE80840FFF78CBE003C01402F
:102FE00068330020084A08B5536911680B4003F0A4
:102FF0001003536123B1054A136A0BB1506A984715
:10300000BDE80840FFF776BE003C01406833002071
:10301000174B10B55C691A68144004F478725A6151
:10302000A30604D5134A936A0BB1D06A9847600689
:1030300004D5104A136B0BB1506B9847210604D589
:103040000C4A936B0BB1D06B9847E20504D5094A43
:10305000136C0BB1506C9847A30504D5054A936CCB
:103060000BB1D06C9847BDE81040FFF743BE00BFDE
:10307000003C0140683300201A4B10B55C691A68A7
:10308000144004F47C425A61620504D5164A136D5B
:103090000BB1506D9847230504D5134A936D0BB1BE
:1030A000D06D9847E00404D50F4A136E0BB1506EF3
:1030B0009847A10404D50C4A936E0BB1D06E984783
:1030C000620404D5084A136F0BB1506F984723046C
:1030D00004D5054A936F0BB1D06F9847BDE81040F7
:1030E000FFF708BE003C014068330020062108B508
:1030F0000846FFF7CBFA06210720FFF7C7FA06219B
:103100000820FFF7C3FA06210920FFF7BFFA0621BE
:103110000A20FFF7BBFA06211720FFF7B7FA0621AE
:103120002820BDE80840FFF7B1BA000008B5FFF756
:1031300049FE00F00BF8FDF761FFFDF73BFEFFF7DE
:10314000C7FDBDE80840FFF7ABBC00000023044901
:103150001A465A50C8180833802B4260F9D170477C
:1031600068330020034611F8012B03F8012B002AD5
:10317000F9D17047121012131211000053544D333D
:1031800032463F3F3F000000000000007C31000855
:103190003F00000013040000B83100083F000000A9
:1031A00019040000C23100083F00000021040000A3
:1031B000CC3100083F00000053544D3332463430C8
:1031C000780053544D3332463432780053544D33E3
:1031D0003246343436585800000000002D0D0008E7
:1031E000190D0008550D0008410D00084D0D00088F
:1031F000390D0008250D0008110D0008B10D00085B
:1032000000000000010000000000000002000000BB
:10321000000000004D0F0008B50F000840004000FE
:10322000342E0020442E0020020000000000000088
:103230000300000000000000F90F0008000000007B
:1032400010000000542E00200000000001000000CB
:1032500000000000F83000200101020025424F412B
:10326000524425002553455249414C25004D617477
:10327000656B463430352D5354440030313233348D
:10328000353637383941424344454600417264750A
:1032900050696C6F740025424F415244252D424CB9
:1032A00000000000391A0008A5180008B90E00082F
:1032B0001D1A000843000000BC3200080902430048
:1032C000020100C0320904000001020201000524CD
:1032D0000010010524010001042402020524060057
:1032E00001070582030800FF09040100020A00002B
:1032F00000070501024000000705810240000000B0
:103300001200000008330008120110010200004002
:103310008304405700020102030100000403090472
:10332000004000000040000000400000004000009D
:103330000000010000000200000002000000020086
:103340000000020000000200000002000000020075
:10335000000000004111000821140008CD140008ED
:10336000400040005831002058310020010000008A
:1033700068310020800000004001000003000000D0
:103380006D61696E00000000A033000870310020FC
:103390006833002001000000C92A00080000000076
:1033A00069646C65000000000000801200000000ED
:1033B000AAAAAAAA00000000FFBF000000000000A7
:1033C00000A00A000000040000000000AAAAAAAAA7
:1033D00000000000FFFD00000000000000000000F1
:1033E0000000000000000000AAAAAAAA0000000035
:1033F000FFFF0000000000000000000000000000CF
:1034000000000000AAAAAAAA00000000FFFF000016
:1034100000000000000000000000000000000000AC
:10342000AAAAAAAA00000000FFFF000000000000F6
:10343000000000000000000000000000AAAAAAAAE4
:1034400000000000FFFF000000000000000000007E
:103450000000000000000000AAAAAAAA00000000C4
:10346000FFFF00000000000000000000000000005E
:10347000000000000A00000000000000030000003F
:10348000000000000000000000000000000000003C
:10349000000000000000000000000000000000002C
:1034A0000000000000000000FF009600000000087F
:1034B000040000001C3300080000000000000000B1
:1034C00000000000000000000000000000000000FC
:00000001FF
